:1000000027C04BC04AC049C048C059C546C045C0BA
:1000100044C043C042C041C040C03FC03EC00102D6
:10002000000000000000000001020408102020046D
:100030001008020202020202020202020000000094
:1000400036000000000038000000000037000B01FF
:1000500011241FBECFE5D2E0DEBFCDBF10E0A0E689
:10006000B0E0E2E2F2E102C005900D92A236B107E3
:10007000D9F720E0A2E6B0E001C01D92A23AB20793
:10008000E1F710E0C0E5D0E003C02297FE01C3D83D
:10009000CE34D107D1F76DD6C2C8B2CF84E890E094
:1000A000ABD361E080916000CDD58FE790E09DD328
:1000B00040E050E060EB72E48FE790E0EAC149D5A0
:1000C000609368007093690080936A0090936B005E
:1000D00060E770E08FE790E03DD1019771F560E750
:1000E00070E08FE790E002D220E030E543EC57E487
:1000F000B0D620E030E040E05FE347D67BD720E099
:1001000030E040E251E4A5D660936C0070936D003E
:1001100080936E0090936F0060E770E08FE790E04F
:10012000DAD190937A0080937900892B11F061E005
:1001300001C060E080916000BED580917D0090910B
:100140007E00019779F440917B0050917C0060E73C
:1001500070E08FE790E0FFD2019721F410927E00CB
:1001600010927D0085E690E081D4882321F1809172
:10017000680090916900A0916A00B0916B00809333
:10018000750090937600A0937700B093780081E09B
:1001900090E090937E0080937D0090937C0080930C
:1001A0007B0060E770E08FE790E0D1D166E970E016
:1001B00080E090E0FED482E690E058D4882331F1CC
:1001C0008091680090916900A0916A00B0916B00E5
:1001D0008093750090937600A0937700B093780099
:1001E00081E090E090937E0080937D0082E090E03B
:1001F00090937C0080937B0060E770E08FE790E055
:1002000028D266E970E080E090E0D3D464E170E049
:1002100080E090E0CEC48FE790E00AD041E063E058
:1002200085E690E000D441E064E082E690E0FBC324
:10023000CF93DF93EC0184E890E0DED281E090E0A0
:100240009C838B83DF91CF910895EF92FF920F9360
:100250001F93CF93DF9300D000D01F92CDB7DEB7AE
:100260007C01FB01CA01B9018E010F5F1F4F25E020
:10027000D8011D922A95E9F7E130F10511F021E04E
:1002800001C021E12B83D7012C9121FF02C030E86E
:100290003C8322FF03C03C8134603C8323FF03C0C6
:1002A0003C8132603C8324FF03C03C8138603C8346
:1002B00025FF03C03C8130623C833C8130613C833C
:1002C00026FF02C030E43D8327FF03C02D81206854
:1002D0002D8320E030E04AE754E4319739F42ED7FB
:1002E00020E030E041E653E450D506C027D720E0B7
:1002F00030E041E653E448D520E030E040E850E407
:100300001DD72FE632E143E052E4A3D50AD67F732E
:1003100079836A8360E684E890E06FD27E01B6E07C
:10032000EB0EF11CF80161918F0184E890E06BD233
:100330000E151F05B9F784E890E071D20F900F9069
:100340000F900F900F90DF91CF911F910F91FF9021
:10035000EF9008950F931F93CF93DF93EB0185E008
:10036000FB0111928A95E9F745E060E684E890E0A8
:1003700063D284E890E07CD2882371F08E01C0E0E3
:10038000D0E084E890E06AD2F80181938F01219651
:10039000C530D105B1F703C080E090E002C081E034
:1003A00090E0DF91CF911F910F910895AF92BF928E
:1003B000CF92DF92EF92FF920F931F93CF93DF9331
:1003C00000D000D01F92CDB7DEB78C016A017B014F
:1003D000CB01BA0160537242894F9F4FCED520E0C6
:1003E00034E244E759E435D59B01AC0161E070E0AB
:1003F000C8012BDF6EE170E080E090E0DAD3BE014F
:100400006F5F7F4FC801A6DF019731F4AC80A294E3
:100410008FE0A822B12C02C0A12CB12CC701B601DB
:10042000605D7D4D86409109A8D520E034E244E727
:1004300059E40FD59B01AC0160E070E0C80105DF15
:100440006EE170E080E090E0B4D3BE016F5F7F4F5B
:10045000C80180DF019759F42C8122952F7030E07C
:1004600081E090E0A216B30624F080E002C080E0B4
:1004700090E00F900F900F900F900F90DF91CF9121
:100480001F910F91FF90EF90DF90CF90BF90AF90B2
:100490000895CF92DF92EF92FF92CF93DF93EC011A
:1004A0006A017B0120E034E244E759E4C701B60168
:1004B00045D637D5AB01BC01CE0178DF9C838B8359
:1004C000A7019601BC01CE01DF91CF91FF90EF9083
:1004D000DF90CF90BACEFB018281992787FD90955E
:1004E000892F881F8827881F90E00895FB01DC0171
:1004F00013968D919C911497608121816F7370E0A8
:10050000762F6627620F711D019781F4882777FD8A
:100510008095982F3DE0660F771F881F991F3A95A9
:10052000D1F7685E7E46834091090FC0882777FD2A
:100530008095982F2DE0660F771F881F991F2A95A9
:10054000D1F7685171498C4F9F4F19D50895EF929B
:10055000FF920F931F93CF93DF938C01EB01C6DFC4
:1005600020E030E040EC57E410D420E034E244E7EF
:1005700059E46FD420E034E244E759E4DFD520E0C9
:100580003AEB4BE558E401D420E030E040E850E499
:10059000D5D520E030E040E058E3D0D5C2D469831F
:1005A0007F737064788380ED8A831B82F801808179
:1005B00081FF02C080E88B83F801808182FF03C045
:1005C0008B8184608B83F801808183FF03C08B81E2
:1005D00082608B83F801808184FF03C08B818860F7
:1005E0008B83F801808185FF03C08B8180628B83C0
:1005F0008B8180618B831C82F801808186FF02C021
:1006000080E48C83F801808187FF03C08C8180683F
:100610008C8360E684E890E0F0D0E12CF12C6991C5
:1006200084E890E0F0D0FFEFEF1AFF0A85E0E816CB
:10063000F104A9F784E890E0F2D081E090E0F801BD
:1006400094838383DF91CF911F910F91FF90EF905F
:100650000895EF92FF920F931F93CF93DF938C0136
:10066000EB0144DF20E030E040EC57E48DD320E0A4
:1006700034E244E759E4EDD320E034E244E759E4BE
:100680005DD520E03AEB4BE558E47FD320E030E045
:1006900040E850E453D520E030E040E058E34ED548
:1006A00040D469837F737064788380E58A831B827A
:1006B000F801808181FF02C080E88B83F80180818E
:1006C00082FF03C08B8184608B83F801808183FF6C
:1006D00003C08B8182608B83F801808184FF03C01B
:1006E0008B8188608B83F801808185FF03C08B81BB
:1006F00080628B838B8180618B831C82F801808177
:1007000086FF02C080E48C83F801808187FF03C0EC
:100710008C8180688C8360E684E890E06ED0E12C68
:10072000F12C699184E890E06ED0FFEFEF1AFF0A98
:1007300085E0E816F104A9F784E890E070D081E044
:1007400090E0F80194838383DF91CF911F910F9103
:10075000FF90EF9008950F931F93CF93DF93EC01D9
:100760008B01FB01808187FF3BC086FF21C04130A8
:10077000510569F440E050E06FEA72E4CE0189DE91
:10078000B801CE01E7DDB801CE01E1DE0FC0423095
:10079000510551F740E050E068ED72E4CE0179DE9A
:1007A000B801CE01D7DDB801CE0153DF80E017C01C
:1007B000CE019CDE20E030E543EC57E44AD320E054
:1007C00030E040E05FE3E1D215D420E030E040E2E9
:1007D00051E43FD3AB01BC01CE015BDE81E090E090
:1007E000DF91CF911F910F910895FC0120812F611E
:1007F0002F792F772083089541C010928700660FCC
:10080000609388000895E0918700E03138F4EF5F4D
:10081000E0938700F0E0E857FF4F60830895609110
:1008200087006F5F88E890E0F5D010928700811113
:1008300001C02FC080E0089510928600409385008B
:10084000660F61606093880061E0640F88E890E063
:10085000E1D0811101C01DC080E00895E0918600C3
:10086000EF5FE0938600F0E0E857FF4F8081089546
:100870008091850090918600891B0895C09AC29A44
:10088000BA9AB89A8FEF8FB98AE28DB980EF8EB994
:1008900008958091980008958EB98BE200C000C041
:1008A00000008DB9B29BFECF00C000C08DB9769B11
:1008B000F5CF00C000C000008FB19FEF9FB9B89A7C
:1008C0000895C29AC29BFECF00C000C00000C0982D
:1008D00000C000C0C298C09A779905C083E0809399
:1008E000980080E0089581E00895C098C29AB29B74
:1008F000FECF00C000C0C09A00C000C000009EB182
:10090000892F807295FD04C094E09093980008951B
:1009100081E00895AF92BF92CF92DF92EF92FF9263
:100920000F931F93CF93DF93EC01C62E8091980015
:10093000816080939800988190FD03C082608093CD
:100940009800BFDF982F882309F458C0FC2C8E0133
:10095000BB24BA94AA24A394209198002370C801C0
:100960000196222371F1C298D82EE92EF8018081D8
:100970008FB980EF91DFB8988EEF8EDF20919800CD
:1009800080FF0AC0922F917020FF04C081E0809305
:10099000980033C082E00EC0822F8570843069F4E5
:1009A000888181608883A09298008BDF982F8111C5
:1009B00018C08AE08093980021C02E7F2093980071
:1009C00013C0B898D82EE92E80EF66DFF801808337
:1009D000F1E0FF1202C0BFB801C01FB88EEF5CDFAC
:1009E00003C0FC2CDC2EED2EFA9419F00D2D1E2DDB
:1009F000B3CF7BDF91E0811101C090E0892FDF91BF
:100A0000CF911F910F91FF90EF90DF90CF90BF900B
:100A1000AF900895109298007DCF21E0FC012183D2
:100A200061E0808148C10F931F93CF93DF931F92A2
:100A3000CDB7DEB78C01862FF801608360E0498373
:100A400001D14981411103C0F801118202C0C801DE
:100A5000E4DFF80112828181811102C081E082838A
:100A60000F90DF91CF911F910F910895CF93DF9356
:100A7000EC018A8180FF02C0826001C08D7F8A8381
:100A800088814ED1298130E04A818217930711F481
:100A90004E7F01C041604A834A81242F30E0C90162
:100AA000959587958227932780FF02C0446001C0F7
:100AB0004B7F4A838A818170DF91CF9108951F9285
:100AC0000F920FB60F9211242F933F938F939F9302
:100AD000AF93BF9380919A0090919B00A0919C004E
:100AE000B0919D003091990020E3230F2D3720F421
:100AF0004096A11DB11D05C023EB230F4196A11DFA
:100B0000B11D2093990080939A0090939B00A0932D
:100B10009C00B0939D0080919E0090919F00A091B9
:100B2000A000B091A1000196A11DB11D80939E006F
:100B300090939F00A093A000B093A100BF91AF91AC
:100B40009F918F913F912F910F900FBE0F901F900B
:100B500018952FB7F89460919A0070919B0080913E
:100B60009C0090919D002FBF08953FB7F89480910D
:100B70009E0090919F00A091A000B091A10022B78B
:100B800008B601FE05C02F3F19F00196A11DB11D49
:100B90003FBF6627782F892F9A2F620F711D811D05
:100BA000911D46E0660F771F881F991F4A95D1F760
:100BB0000895CF92DF92EF92FF92CF93DF936B0174
:100BC0007C01D3DFEB01C114D104E104F10479F01D
:100BD000DAD0CBDF6C1B7D0B683E7340A0F381E065
:100BE000C81AD108E108F108C851DC4FECCFDF91F9
:100BF000CF91FF90EF90DF90CF90089578948AB5D1
:100C000082608ABD8AB581608ABD83B7826083BFF6
:100C100083B7816083BF89B7826089BF80B78260F4
:100C200080BF329A319A309A379A0895813019F0FC
:100C3000823021F008958AB58F7702C08AB58F7D02
:100C40008ABD0895CF93DF9390E0FC01E85DFF4FEC
:100C50002491FC01EE5CFF4F8491882349F190E0E0
:100C6000880F991FFC01E85BFF4FA591B4918E5B43
:100C70009F4FFC01C591D4919FB7611108C0F894B2
:100C80008C91209582238C93888182230AC06230C4
:100C900051F4F8948C91322F309583238C93888172
:100CA000822B888304C0F8948C91822B8C939FBFF5
:100CB000DF91CF9108950F931F93CF93DF931F92EE
:100CC000CDB7DEB7282F30E0F901E25EFF4F849107
:100CD000F901E85DFF4F1491F901EE5CFF4F0491BB
:100CE0000023C1F0882319F06983A0DF6981E02F18
:100CF000F0E0EE0FFF1FEE5BFF4FA591B4919FB7A1
:100D0000F8948C91611103C01095812301C0812B4F
:100D10008C939FBF0F90DF91CF911F910F910895FA
:100D2000CF93DF93282F30E0F901E25EFF4F8491EB
:100D3000F901E85DFF4FD491F901EE5CFF4FC491DA
:100D4000CC2389F0811172DFEC2FF0E0EE0FFF1F52
:100D5000E45CFF4FA591B4912C912D2381E090E0AC
:100D600021F480E002C080E090E0DF91CF9108950F
:100D7000089544DFFDDF92D9C0E0D0E0A0D92097EC
:100D8000E9F33ED9FBCF08955058BB27AA270ED0D0
:100D900084C175D130F07AD120F031F49F3F11F445
:100DA0001EF46AC10EF4E095E7FB37C1E92F86D146
:100DB00080F3BA17620773078407950718F071F478
:100DC0009EF5B5C10EF4E0950B2EBA2FA02D0B01A8
:100DD000B90190010C01CA01A0011124FF27591B80
:100DE00099F0593F50F4503E68F11A16F040A22F86
:100DF000232F342F4427585FF3CF469537952795F7
:100E0000A795F0405395C9F77EF41F16BA0B620BF5
:100E1000730B840BBAF09150A1F0FF0FBB1F661F3C
:100E2000771F881FC2F70EC0BA0F621F731F841F7F
:100E300048F4879577956795B795F7959E3F08F0A5
:100E4000B3CF9395880F08F09927EE0F9795879564
:100E500008950CD022C11AD140F011D130F021F404
:100E60005F3F19F0DAC0511163C106C127D198F371
:100E70009923C9F35523B1F3951B550BBB27AA271B
:100E800062177307840738F09F5F5F4F220F331F8D
:100E9000441FAA1FA9F333D00E2E3AF0E0E830D059
:100EA00091505040E695001CCAF729D0FE2F27D05C
:100EB000660F771F881FBB1F261737074807AB072A
:100EC000B0E809F0BB0B802DBF01FF2793585F4F9F
:100ED0002AF09E3F510568F0A0C02AC15F3FECF3A5
:100EE000983EDCF3869577956795B795F7959F5F64
:100EF000C9F7880F911D9695879597F90895E1E0B8
:100F0000660F771F881FBB1F621773078407BA0716
:100F100020F0621B730B840BBA0BEE1F88F7E09571
:100F20000895D4D088F09F5790F0B92F9927B751E2
:100F3000A0F0D1F0660F771F881F991F1AF0BA959D
:100F4000C9F712C0B13081F0F2D0B1E00895EFC01E
:100F5000672F782F8827B85F39F0B93FCCF3869593
:100F600077956795B395D9F73EF4909580957095F0
:100F700061957F4F8F4F9F4F0895E89409C097FB6D
:100F80003EF490958095709561957F4F8F4F9F4F60
:100F90009923A9F0F92F96E9BB279395F6958795A4
:100FA00077956795B795F111F8CFFAF4BB0F11F467
:100FB00060FF1BC06F5F7F4F8F4F9F4F16C088230E
:100FC00011F096E911C0772321F09EE8872F762F44
:100FD00005C0662371F096E8862F70E060E02AF085
:100FE0009A95660F771F881FDAF7880F9695879571
:100FF00097F9089585D080F09F3740F491110EF055
:1010000097C060E070E080E89FEB089526F41B161F
:10101000611D711D811D07C021C097F99F6780E880
:1010200070E060E00895882371F4772321F09850F0
:10103000872B762F07C0662311F499270DC0905196
:10104000862B70E060E02AF09A95660F771F881F64
:10105000DAF7880F9695879597F908959F3F31F0B5
:10106000915020F4879577956795B795880F911DD6
:101070009695879597F908959FEF80EC0895002441
:101080000A941616170618060906089500240A94ED
:1010900012161306140605060895092E0394000C73
:1010A00011F4882352F0BB0F40F4BF2B11F460FF02
:1010B00004C06F5F7F4F8F4F9F4F089557FD90582B
:1010C000440F551F59F05F3F71F04795880F97FB0C
:1010D000991F61F09F3F79F08795089512161306C6
:1010E0001406551FF2CF4695F1DF08C016161706F5
:1010F0001806991FF1CF869571056105089408952A
:10110000E5DFA0F0BEE7B91788F4BB279F3860F48D
:101110001616B11D672F782F8827985FF7CF869511
:1011200077956795B11D93959639C8F30895E8941E
:10113000BB2766277727CB0197F908950AD0ADCF53
:101140009EDF28F0A3DF18F0952309F066CF94CF37
:10115000EFCFB4DFA8F39923D9F35523C9F3950F43
:1011600050E0551FAA27EE27FF27BB27002408942D
:10117000679520F4E20FF31FB41F0A1E220F331FDE
:10118000441FAA1F6695A9F7779530F4F30FB41F93
:101190000A1E121E08F46395330F441FAA1F221F54
:1011A000769599F7879520F4B40F0A1E121E631FD7
:1011B000440FAA1F221F331F8695A9F7862F712D72
:1011C000602D11249F5750408AF0E1F088234AF0A7
:1011D000EE0FFF1FBB1F661F771F881F91505040E7
:1011E000A9F79E3F510570F018CFA2CF5F3FECF3F7
:1011F000983EDCF3869577956795B795F795E795D3
:101200009F5FC1F7FE2B880F911D9695879597F9E3
:101210000895EE0FFF1F0590F491E02D0994F894C6
:02122000FFCFFE
:021222000100C9
:00000001FF
